Archive member included to satisfy reference by file (symbol)

c:/program files (x86)/gnu_arm_embedded_toolchain/bin/../lib/gcc/arm-none-eabi/9.3.1/thumb/v6-m/nofp\libgcc.a(_udivsi3.o)
                              Output/printf.o (__aeabi_uidiv)
c:/program files (x86)/gnu_arm_embedded_toolchain/bin/../lib/gcc/arm-none-eabi/9.3.1/thumb/v6-m/nofp\libgcc.a(_divsi3.o)
                              Output/PdbPowerMonitor.o (__aeabi_idiv)
c:/program files (x86)/gnu_arm_embedded_toolchain/bin/../lib/gcc/arm-none-eabi/9.3.1/thumb/v6-m/nofp\libgcc.a(_dvmd_tls.o)
                              c:/program files (x86)/gnu_arm_embedded_toolchain/bin/../lib/gcc/arm-none-eabi/9.3.1/thumb/v6-m/nofp\libgcc.a(_udivsi3.o) (__aeabi_idiv0)
c:/program files (x86)/gnu_arm_embedded_toolchain/bin/../lib/gcc/arm-none-eabi/9.3.1/thumb/v6-m/nofp\libgcc.a(_aeabi_uldivmod.o)
                              Output/printf.o (__aeabi_uldivmod)
c:/program files (x86)/gnu_arm_embedded_toolchain/bin/../lib/gcc/arm-none-eabi/9.3.1/thumb/v6-m/nofp\libgcc.a(_udivmoddi4.o)
                              c:/program files (x86)/gnu_arm_embedded_toolchain/bin/../lib/gcc/arm-none-eabi/9.3.1/thumb/v6-m/nofp\libgcc.a(_aeabi_uldivmod.o) (__udivmoddi4)
c:/program files (x86)/gnu_arm_embedded_toolchain/bin/../lib/gcc/arm-none-eabi/9.3.1/thumb/v6-m/nofp\libgcc.a(_clzdi2.o)
                              c:/program files (x86)/gnu_arm_embedded_toolchain/bin/../lib/gcc/arm-none-eabi/9.3.1/thumb/v6-m/nofp\libgcc.a(_udivmoddi4.o) (__clzdi2)
c:/program files (x86)/gnu_arm_embedded_toolchain/bin/../lib/gcc/arm-none-eabi/9.3.1/thumb/v6-m/nofp\libgcc.a(_clzsi2.o)
                              c:/program files (x86)/gnu_arm_embedded_toolchain/bin/../lib/gcc/arm-none-eabi/9.3.1/thumb/v6-m/nofp\libgcc.a(_clzdi2.o) (__clzsi2)
c:/program files (x86)/gnu_arm_embedded_toolchain/bin/../lib/gcc/arm-none-eabi/9.3.1/../../../../arm-none-eabi/lib/thumb/v6-m/nofp\libc_nano.a(lib_a-exit.o)
                              c:/program files (x86)/gnu_arm_embedded_toolchain/bin/../lib/gcc/arm-none-eabi/9.3.1/../../../../arm-none-eabi/lib/thumb/v6-m/nofp/crt0.o (exit)
c:/program files (x86)/gnu_arm_embedded_toolchain/bin/../lib/gcc/arm-none-eabi/9.3.1/../../../../arm-none-eabi/lib/thumb/v6-m/nofp\libc_nano.a(lib_a-impure.o)
                              c:/program files (x86)/gnu_arm_embedded_toolchain/bin/../lib/gcc/arm-none-eabi/9.3.1/../../../../arm-none-eabi/lib/thumb/v6-m/nofp\libc_nano.a(lib_a-exit.o) (_global_impure_ptr)
c:/program files (x86)/gnu_arm_embedded_toolchain/bin/../lib/gcc/arm-none-eabi/9.3.1/../../../../arm-none-eabi/lib/thumb/v6-m/nofp\libc_nano.a(lib_a-init.o)
                              c:/program files (x86)/gnu_arm_embedded_toolchain/bin/../lib/gcc/arm-none-eabi/9.3.1/../../../../arm-none-eabi/lib/thumb/v6-m/nofp/crt0.o (__libc_init_array)
c:/program files (x86)/gnu_arm_embedded_toolchain/bin/../lib/gcc/arm-none-eabi/9.3.1/../../../../arm-none-eabi/lib/thumb/v6-m/nofp\libc_nano.a(lib_a-memset.o)
                              c:/program files (x86)/gnu_arm_embedded_toolchain/bin/../lib/gcc/arm-none-eabi/9.3.1/../../../../arm-none-eabi/lib/thumb/v6-m/nofp/crt0.o (memset)

Allocating common symbols
Common symbol       size              file

PdbPwrMonData       0x14              Output/PdbPowerMonitor.o
SysTickCallbacks    0x10              Output/SYSTEM_Driver.o
_MCAN0_message_ram  0x100             Output/MCAN_Driver.o
lastStatusMessage   0x4               Output/CommSystem.o

Discarded input sections

 .text          0x00000000        0x0 c:/program files (x86)/gnu_arm_embedded_toolchain/bin/../lib/gcc/arm-none-eabi/9.3.1/thumb/v6-m/nofp/crti.o
 .data          0x00000000        0x0 c:/program files (x86)/gnu_arm_embedded_toolchain/bin/../lib/gcc/arm-none-eabi/9.3.1/thumb/v6-m/nofp/crti.o
 .bss           0x00000000        0x0 c:/program files (x86)/gnu_arm_embedded_toolchain/bin/../lib/gcc/arm-none-eabi/9.3.1/thumb/v6-m/nofp/crti.o
 .data          0x00000000        0x4 c:/program files (x86)/gnu_arm_embedded_toolchain/bin/../lib/gcc/arm-none-eabi/9.3.1/thumb/v6-m/nofp/crtbegin.o
 .text          0x00000000       0x80 c:/program files (x86)/gnu_arm_embedded_toolchain/bin/../lib/gcc/arm-none-eabi/9.3.1/../../../../arm-none-eabi/lib/thumb/v6-m/nofp/crt0.o
 .data          0x00000000        0x0 c:/program files (x86)/gnu_arm_embedded_toolchain/bin/../lib/gcc/arm-none-eabi/9.3.1/../../../../arm-none-eabi/lib/thumb/v6-m/nofp/crt0.o
 .bss           0x00000000        0x0 c:/program files (x86)/gnu_arm_embedded_toolchain/bin/../lib/gcc/arm-none-eabi/9.3.1/../../../../arm-none-eabi/lib/thumb/v6-m/nofp/crt0.o
 .ARM.extab     0x00000000        0x0 c:/program files (x86)/gnu_arm_embedded_toolchain/bin/../lib/gcc/arm-none-eabi/9.3.1/../../../../arm-none-eabi/lib/thumb/v6-m/nofp/crt0.o
 .ARM.exidx     0x00000000       0x10 c:/program files (x86)/gnu_arm_embedded_toolchain/bin/../lib/gcc/arm-none-eabi/9.3.1/../../../../arm-none-eabi/lib/thumb/v6-m/nofp/crt0.o
 .ARM.attributes
                0x00000000       0x1b c:/program files (x86)/gnu_arm_embedded_toolchain/bin/../lib/gcc/arm-none-eabi/9.3.1/../../../../arm-none-eabi/lib/thumb/v6-m/nofp/crt0.o
 .group         0x00000000        0xc Output/startup_samc21.o
 .group         0x00000000        0xc Output/startup_samc21.o
 .group         0x00000000        0xc Output/startup_samc21.o
 .group         0x00000000        0xc Output/startup_samc21.o
 .group         0x00000000        0xc Output/startup_samc21.o
 .group         0x00000000        0xc Output/startup_samc21.o
 .group         0x00000000        0xc Output/startup_samc21.o
Memory Configuration

Name             Origin             Length             Attributes
rom              0x00000000         0x00040000         xr
ram              0x20000000         0x00008000         xrw
*default*        0x00000000         0xffffffff

Linker script and memory map

LOAD c:/program files (x86)/gnu_arm_embedded_toolchain/bin/../lib/gcc/arm-none-eabi/9.3.1/thumb/v6-m/nofp/crti.o
LOAD c:/program files (x86)/gnu_arm_embedded_toolchain/bin/../lib/gcc/arm-none-eabi/9.3.1/thumb/v6-m/nofp/crtbegin.o
LOAD c:/program files (x86)/gnu_arm_embedded_toolchain/bin/../lib/gcc/arm-none-eabi/9.3.1/../../../../arm-none-eabi/lib/thumb/v6-m/nofp/crt0.o
                0x00000800                STACK_SIZE = DEFINED (STACK_SIZE)?STACK_SIZE:DEFINED (__stack_size__)?__stack_size__:0x800

.text           0x00000000     0x150c
                0x00000000                . = ALIGN (0x4)
                0x00000000                _sfixed = .
 *(.vectors .vectors.*)
 .vectors       0x00000000       0xbc Output/startup_samc21.o
                0x00000000                exception_table
 *(.text .text.* .gnu.linkonce.t.*)
 .text          0x000000bc       0x48 c:/program files (x86)/gnu_arm_embedded_toolchain/bin/../lib/gcc/arm-none-eabi/9.3.1/thumb/v6-m/nofp/crtbegin.o
 .text.Dummy_Handler
                0x00000104        0x2 Output/startup_samc21.o
                0x00000104                SVCall_Handler
                0x00000104                DMAC_Handler
                0x00000104                HardFault_Handler
                0x00000104                TC2_Handler
                0x00000104                AC_Handler
                0x00000104                PendSV_Handler
                0x00000104                NonMaskableInt_Handler
                0x00000104                TCC1_Handler
                0x00000104                TCC0_Handler
                0x00000104                RTC_Handler
                0x00000104                ADC1_Handler
                0x00000104                WDT_Handler
                0x00000104                CAN0_Handler
                0x00000104                TC4_Handler
                0x00000104                TC1_Handler
                0x00000104                TC3_Handler
                0x00000104                SDADC_Handler
                0x00000104                Dummy_Handler
                0x00000104                CAN1_Handler
                0x00000104                ADC0_Handler
                0x00000104                TSENS_Handler
                0x00000104                TCC2_Handler
                0x00000104                EVSYS_Handler
                0x00000104                NVMCTRL_Handler
                0x00000104                SYSTEM_Handler
                0x00000104                DAC_Handler
                0x00000104                PTC_Handler
                0x00000104                FREQM_Handler
                0x00000104                TC0_Handler
 *fill*         0x00000106        0x2 
 .text.Reset_Handler
                0x00000108       0x5c Output/startup_samc21.o
                0x00000108                Reset_Handler
 .text.SystemInit
                0x00000164       0x2c Output/system_samc21.o
                0x00000164                SystemInit
 .text.IVREF_Setup
                0x00000190       0x1c Output/ADC_Driver.o
                0x00000190                IVREF_Setup
 .text.ADC_Initialize
                0x000001ac      0x144 Output/ADC_Driver.o
                0x000001ac                ADC_Initialize
 .text.ADC_SetSingleEndedChannel
                0x000002f0       0x1c Output/ADC_Driver.o
                0x000002f0                ADC_SetSingleEndedChannel
 .text.ADC_StartConversion
                0x0000030c       0x20 Output/ADC_Driver.o
                0x0000030c                ADC_StartConversion
 .text.GPIO_SetPinMode
                0x0000032c       0x9e Output/GPIO_Driver.o
                0x0000032c                GPIO_SetPinMode
 .text.GPIO_SetPinMux
                0x000003ca       0x52 Output/GPIO_Driver.o
                0x000003ca                GPIO_SetPinMux
 .text.GPIO_GetPinState
                0x0000041c       0x1c Output/GPIO_Driver.o
                0x0000041c                GPIO_GetPinState
 .text.MCAN_Initialize
                0x00000438      0x1c4 Output/MCAN_Driver.o
                0x00000438                MCAN_Initialize
 .text.MCAN_ChangeMode
                0x000005fc       0x88 Output/MCAN_Driver.o
                0x000005fc                MCAN_ChangeMode
 .text.MCAN_ReadFIFOMessage
                0x00000684       0xaa Output/MCAN_Driver.o
                0x00000684                MCAN_ReadFIFOMessage
 *fill*         0x0000072e        0x2 
 .text.MCAN_TransmitMessageFIFO
                0x00000730       0x6c Output/MCAN_Driver.o
                0x00000730                MCAN_TransmitMessageFIFO
 .text.SERCOM0_Handler
                0x0000079c       0x18 Output/SERCOM_Driver.o
                0x0000079c                SERCOM0_Handler
 .text.SERCOM1_Handler
                0x000007b4       0x18 Output/SERCOM_Driver.o
                0x000007b4                SERCOM1_Handler
 .text.SERCOM2_Handler
                0x000007cc       0x18 Output/SERCOM_Driver.o
                0x000007cc                SERCOM2_Handler
 .text.SERCOM3_Handler
                0x000007e4       0x18 Output/SERCOM_Driver.o
                0x000007e4                SERCOM3_Handler
 .text.SERCOM4_Handler
                0x000007fc       0x18 Output/SERCOM_Driver.o
                0x000007fc                SERCOM4_Handler
 .text.SERCOM5_Handler
                0x00000814       0x18 Output/SERCOM_Driver.o
                0x00000814                SERCOM5_Handler
 .text.SYSTEM_InitializeClocks
                0x0000082c       0xa0 Output/SYSTEM_Driver.o
                0x0000082c                SYSTEM_InitializeClocks
 .text.SYSTEM_IsClockSourceAvailable
                0x000008cc       0x14 Output/SYSTEM_Driver.o
                0x000008cc                SYSTEM_IsClockSourceAvailable
 .text.SYSTEM_InitalizeSysTick
                0x000008e0       0x40 Output/SYSTEM_Driver.o
                0x000008e0                SYSTEM_InitalizeSysTick
 .text.SYSTEM_GetSysTickCount
                0x00000920        0xc Output/SYSTEM_Driver.o
                0x00000920                SYSTEM_GetSysTickCount
 .text.SysTick_Handler
                0x0000092c       0x2c Output/SYSTEM_Driver.o
                0x0000092c                SysTick_Handler
 .text.main     0x00000958       0x22 Output/main.o
                0x00000958                main
 *fill*         0x0000097a        0x2 
 .text.CommSystem_Initialize
                0x0000097c       0x40 Output/CommSystem.o
                0x0000097c                CommSystem_Initialize
 .text.CommSystem_SendStatus
                0x000009bc       0x34 Output/CommSystem.o
                0x000009bc                CommSystem_SendStatus
 .text.CommSystem_Task
                0x000009f0       0x5c Output/CommSystem.o
                0x000009f0                CommSystem_Task
 .text.CommSystem_SendFault
                0x00000a4c       0x2c Output/CommSystem.o
                0x00000a4c                CommSystem_SendFault
 .text.CommSystem_ComposeMessage
                0x00000a78       0x2c Output/CommSystem.o
                0x00000a78                CommSystem_ComposeMessage
 .text.CommSystem_SendData
                0x00000aa4       0x80 Output/CommSystem.o
                0x00000aa4                CommSystem_SendData
 .text.PdbPwrMon_ADC
                0x00000b24      0x1f0 Output/PdbPowerMonitor.o
                0x00000b24                PdbPwrMon_ADC
 .text.PdbPwrMon_GetData
                0x00000d14        0x8 Output/PdbPowerMonitor.o
                0x00000d14                PdbPwrMon_GetData
 .text.PdbPwrMon_eFuseControl
                0x00000d1c       0x90 Output/PdbPowerMonitor.o
                0x00000d1c                PdbPwrMon_eFuseControl
 .text.PdbPwrMon_Initialize
                0x00000dac      0x1b8 Output/PdbPowerMonitor.o
                0x00000dac                PdbPwrMon_Initialize
 .text.PdbPwrMon_FaultControl
                0x00000f64       0xd0 Output/PdbPowerMonitor.o
                0x00000f64                PdbPwrMon_FaultControl
 .text.PdbPwrMon_Task
                0x00001034       0x8c Output/PdbPowerMonitor.o
                0x00001034                PdbPwrMon_Task
 .text.EIC_Handler
                0x000010c0       0xe8 Output/PdbPowerMonitor.o
                0x000010c0                EIC_Handler
 .text          0x000011a8      0x114 c:/program files (x86)/gnu_arm_embedded_toolchain/bin/../lib/gcc/arm-none-eabi/9.3.1/thumb/v6-m/nofp\libgcc.a(_udivsi3.o)
                0x000011a8                __aeabi_uidiv
                0x000011a8                __udivsi3
                0x000012b4                __aeabi_uidivmod
 .text          0x000012bc      0x1d4 c:/program files (x86)/gnu_arm_embedded_toolchain/bin/../lib/gcc/arm-none-eabi/9.3.1/thumb/v6-m/nofp\libgcc.a(_divsi3.o)
                0x000012bc                __divsi3
                0x000012bc                __aeabi_idiv
                0x00001488                __aeabi_idivmod
 .text          0x00001490        0x4 c:/program files (x86)/gnu_arm_embedded_toolchain/bin/../lib/gcc/arm-none-eabi/9.3.1/thumb/v6-m/nofp\libgcc.a(_dvmd_tls.o)
                0x00001490                __aeabi_idiv0
                0x00001490                __aeabi_ldiv0
 .text.__libc_init_array
                0x00001494       0x48 c:/program files (x86)/gnu_arm_embedded_toolchain/bin/../lib/gcc/arm-none-eabi/9.3.1/../../../../arm-none-eabi/lib/thumb/v6-m/nofp\libc_nano.a(lib_a-init.o)
                0x00001494                __libc_init_array
 .text.memset   0x000014dc       0x10 c:/program files (x86)/gnu_arm_embedded_toolchain/bin/../lib/gcc/arm-none-eabi/9.3.1/../../../../arm-none-eabi/lib/thumb/v6-m/nofp\libc_nano.a(lib_a-memset.o)
                0x000014dc                memset
 *(.glue_7t)
 .glue_7t       0x000014ec        0x0 linker stubs
 *(.glue_7)
 .glue_7        0x000014ec        0x0 linker stubs
 *(.rodata .rodata* .gnu.linkonce.r.*)
 *(.ARM.extab* .gnu.linkonce.armextab.*)
                0x000014ec                . = ALIGN (0x4)
 *(.init)
 .init          0x000014ec        0x4 c:/program files (x86)/gnu_arm_embedded_toolchain/bin/../lib/gcc/arm-none-eabi/9.3.1/thumb/v6-m/nofp/crti.o
                0x000014ec                _init
 .init          0x000014f0        0x8 c:/program files (x86)/gnu_arm_embedded_toolchain/bin/../lib/gcc/arm-none-eabi/9.3.1/thumb/v6-m/nofp/crtn.o
                0x000014f8                . = ALIGN (0x4)
                0x000014f8                __preinit_array_start = .
 *(.preinit_array)
                0x000014f8                __preinit_array_end = .
                0x000014f8                . = ALIGN (0x4)
                0x000014f8                __init_array_start = .
 *(SORT_BY_NAME(.init_array.*))
 *(.init_array)
 .init_array    0x000014f8        0x4 c:/program files (x86)/gnu_arm_embedded_toolchain/bin/../lib/gcc/arm-none-eabi/9.3.1/thumb/v6-m/nofp/crtbegin.o
                0x000014fc                __init_array_end = .
                0x000014fc                . = ALIGN (0x4)
 *crtbegin.o(.ctors)
 *(EXCLUDE_FILE(*crtend.o) .ctors)
 *(SORT_BY_NAME(.ctors.*))
 *crtend.o(.ctors)
                0x000014fc                . = ALIGN (0x4)
 *(.fini)
 .fini          0x000014fc        0x4 c:/program files (x86)/gnu_arm_embedded_toolchain/bin/../lib/gcc/arm-none-eabi/9.3.1/thumb/v6-m/nofp/crti.o
                0x000014fc                _fini
 .fini          0x00001500        0x8 c:/program files (x86)/gnu_arm_embedded_toolchain/bin/../lib/gcc/arm-none-eabi/9.3.1/thumb/v6-m/nofp/crtn.o
                0x00001508                . = ALIGN (0x4)
                0x00001508                __fini_array_start = .
 *(.fini_array)
 .fini_array    0x00001508        0x4 c:/program files (x86)/gnu_arm_embedded_toolchain/bin/../lib/gcc/arm-none-eabi/9.3.1/thumb/v6-m/nofp/crtbegin.o
 *(SORT_BY_NAME(.fini_array.*))
                0x0000150c                __fini_array_end = .
 *crtbegin.o(.dtors)
 *(EXCLUDE_FILE(*crtend.o) .dtors)
 *(SORT_BY_NAME(.dtors.*))
 *crtend.o(.dtors)
                0x0000150c                . = ALIGN (0x4)
                0x0000150c                _efixed = .
                [!provide]                PROVIDE (__exidx_start = .)

.vfp11_veneer   0x0000150c        0x0
 .vfp11_veneer  0x0000150c        0x0 linker stubs

.v4_bx          0x0000150c        0x0
 .v4_bx         0x0000150c        0x0 linker stubs

.iplt           0x0000150c        0x0
 .iplt          0x0000150c        0x0 c:/program files (x86)/gnu_arm_embedded_toolchain/bin/../lib/gcc/arm-none-eabi/9.3.1/thumb/v6-m/nofp/crtbegin.o

.igot.plt       0x0000150c        0x0
 .igot.plt      0x0000150c        0x0 c:/program files (x86)/gnu_arm_embedded_toolchain/bin/../lib/gcc/arm-none-eabi/9.3.1/thumb/v6-m/nofp/crtbegin.o

.eh_frame       0x0000150c        0x0
 .eh_frame      0x0000150c        0x0 c:/program files (x86)/gnu_arm_embedded_toolchain/bin/../lib/gcc/arm-none-eabi/9.3.1/thumb/v6-m/nofp/crtbegin.o

.rel.dyn        0x0000150c        0x0
 .rel.iplt      0x0000150c        0x0 c:/program files (x86)/gnu_arm_embedded_toolchain/bin/../lib/gcc/arm-none-eabi/9.3.1/thumb/v6-m/nofp/crtbegin.o

.ARM.exidx
 *(.ARM.exidx* .gnu.linkonce.armexidx.*)
                [!provide]                PROVIDE (__exidx_end = .)
                0x0000150c                . = ALIGN (0x4)
                0x0000150c                _etext = .

.relocate       0x20000000       0x48 load address 0x0000150c
                0x20000000                . = ALIGN (0x4)
                0x20000000                _srelocate = .
 *(.ramfunc .ramfunc.*)
 *(.data .data.*)
 .data.MCAN0    0x20000000       0x28 Output/MCAN_Driver.o
                0x20000000                MCAN0
 .data.SystemClockStatus
                0x20000028        0x4 Output/SYSTEM_Driver.o
 .data.MCAN0_Config
                0x2000002c       0x1c Output/MCAN_Config.o
                0x2000002c                MCAN0_Config
                0x20000048                . = ALIGN (0x4)
                0x20000048                _erelocate = .

.persistent     0x20000048        0x4 load address 0x00001554
                0x20000048                . = ALIGN (0x4)
 *(.persistent .persistent.*)
 .persistent    0x20000048        0x4 Output/system_samc21.o
                0x20000048                SystemCoreClock

.bss            0x2000004c      0x1ac load address 0x00001558
                0x2000004c                . = ALIGN (0x4)
                0x2000004c                _sbss = .
                0x2000004c                _szero = .
 *(.bss .bss.*)
 .bss           0x2000004c       0x1c c:/program files (x86)/gnu_arm_embedded_toolchain/bin/../lib/gcc/arm-none-eabi/9.3.1/thumb/v6-m/nofp/crtbegin.o
 .bss.sercomIsrHandle
                0x20000068       0x18 Output/SERCOM_Driver.o
 .bss.sercomIsrHandler
                0x20000080       0x18 Output/SERCOM_Driver.o
 .bss.SysTickCounter
                0x20000098        0x4 Output/SYSTEM_Driver.o
 .bss.ECUOnline
                0x2000009c        0x1 Output/CommSystem.o
                0x2000009c                ECUOnline
 *fill*         0x2000009d        0x3 
 .bss.datelFaultTime
                0x200000a0        0x4 Output/PdbPowerMonitor.o
                0x200000a0                datelFaultTime
 .bss.datelFaults
                0x200000a4        0x1 Output/PdbPowerMonitor.o
                0x200000a4                datelFaults
 *fill*         0x200000a5        0x3 
 .bss.ecupcFaultTime
                0x200000a8        0x4 Output/PdbPowerMonitor.o
                0x200000a8                ecupcFaultTime
 .bss.ecupcFaults
                0x200000ac        0x1 Output/PdbPowerMonitor.o
                0x200000ac                ecupcFaults
 *fill*         0x200000ad        0x3 
 .bss.invaFaultTime
                0x200000b0        0x4 Output/PdbPowerMonitor.o
                0x200000b0                invaFaultTime
 .bss.invaFaults
                0x200000b4        0x1 Output/PdbPowerMonitor.o
                0x200000b4                invaFaults
 *fill*         0x200000b5        0x3 
 .bss.invfFaultTime
                0x200000b8        0x4 Output/PdbPowerMonitor.o
                0x200000b8                invfFaultTime
 .bss.invfFaults
                0x200000bc        0x1 Output/PdbPowerMonitor.o
                0x200000bc                invfFaults
 *fill*         0x200000bd        0x3 
 .bss.lastAcqTime
                0x200000c0        0x4 Output/PdbPowerMonitor.o
                0x200000c0                lastAcqTime
 .bss.lastExtLedBlinkTime
                0x200000c4        0x4 Output/PdbPowerMonitor.o
                0x200000c4                lastExtLedBlinkTime
 .bss.safamFaultTime
                0x200000c8        0x4 Output/PdbPowerMonitor.o
                0x200000c8                safamFaultTime
 .bss.safamFaults
                0x200000cc        0x1 Output/PdbPowerMonitor.o
                0x200000cc                safamFaults
 *(COMMON)
 *fill*         0x200000cd        0x3 
 COMMON         0x200000d0      0x100 Output/MCAN_Driver.o
                0x200000d0                _MCAN0_message_ram
 COMMON         0x200001d0       0x10 Output/SYSTEM_Driver.o
                0x200001d0                SysTickCallbacks
 COMMON         0x200001e0        0x4 Output/CommSystem.o
                0x200001e0                lastStatusMessage
 COMMON         0x200001e4       0x14 Output/PdbPowerMonitor.o
                0x200001e4                PdbPwrMonData
                0x200001f8                . = ALIGN (0x4)
                0x200001f8                _ebss = .
                0x200001f8                _ezero = .

.stack          0x200001f8      0x800 load address 0x00001704
                0x200001f8                . = ALIGN (0x8)
                0x200001f8                _sstack = .
                0x200009f8                . = (. + STACK_SIZE)
 *fill*         0x200001f8      0x800 
                0x200009f8                . = ALIGN (0x8)
                0x200009f8                _estack = .
                0x200009f8                . = ALIGN (0x4)
                0x200009f8                _end = .
LOAD Output/startup_samc21.o
LOAD Output/system_samc21.o
LOAD Output/fifobuffer.o
LOAD Output/printf.o
LOAD Output/ADC_Driver.o
LOAD Output/GPIO_Driver.o
LOAD Output/MCAN_Driver.o
LOAD Output/SERCOM_Driver.o
LOAD Output/SYSTEM_Driver.o
LOAD Output/MCAN_Config.o
LOAD Output/main.o
LOAD Output/CommSystem.o
LOAD Output/PdbPowerMonitor.o
START GROUP
LOAD c:/program files (x86)/gnu_arm_embedded_toolchain/bin/../lib/gcc/arm-none-eabi/9.3.1/thumb/v6-m/nofp\libgcc.a
LOAD c:/program files (x86)/gnu_arm_embedded_toolchain/bin/../lib/gcc/arm-none-eabi/9.3.1/../../../../arm-none-eabi/lib/thumb/v6-m/nofp\libc_nano.a
END GROUP
START GROUP
LOAD c:/program files (x86)/gnu_arm_embedded_toolchain/bin/../lib/gcc/arm-none-eabi/9.3.1/thumb/v6-m/nofp\libgcc.a
LOAD c:/program files (x86)/gnu_arm_embedded_toolchain/bin/../lib/gcc/arm-none-eabi/9.3.1/../../../../arm-none-eabi/lib/thumb/v6-m/nofp\libc_nano.a
END GROUP
LOAD c:/program files (x86)/gnu_arm_embedded_toolchain/bin/../lib/gcc/arm-none-eabi/9.3.1/thumb/v6-m/nofp/crtend.o
LOAD c:/program files (x86)/gnu_arm_embedded_toolchain/bin/../lib/gcc/arm-none-eabi/9.3.1/thumb/v6-m/nofp/crtn.o
OUTPUT(Output/PDB_Monitoring.elf elf32-littlearm)
LOAD linker stubs

.ARM.attributes
                0x00000000       0x28
 .ARM.attributes
                0x00000000       0x1e c:/program files (x86)/gnu_arm_embedded_toolchain/bin/../lib/gcc/arm-none-eabi/9.3.1/thumb/v6-m/nofp/crti.o
 .ARM.attributes
                0x0000001e       0x2c c:/program files (x86)/gnu_arm_embedded_toolchain/bin/../lib/gcc/arm-none-eabi/9.3.1/thumb/v6-m/nofp/crtbegin.o
 .ARM.attributes
                0x0000004a       0x2c Output/startup_samc21.o
 .ARM.attributes
                0x00000076       0x2c Output/system_samc21.o
 .ARM.attributes
                0x000000a2       0x2c Output/ADC_Driver.o
 .ARM.attributes
                0x000000ce       0x2c Output/GPIO_Driver.o
 .ARM.attributes
                0x000000fa       0x2c Output/MCAN_Driver.o
 .ARM.attributes
                0x00000126       0x2c Output/SERCOM_Driver.o
 .ARM.attributes
                0x00000152       0x2c Output/SYSTEM_Driver.o
 .ARM.attributes
                0x0000017e       0x32 Output/MCAN_Config.o
 .ARM.attributes
                0x000001b0       0x2c Output/main.o
 .ARM.attributes
                0x000001dc       0x2c Output/CommSystem.o
 .ARM.attributes
                0x00000208       0x2c Output/PdbPowerMonitor.o
 .ARM.attributes
                0x00000234       0x1e c:/program files (x86)/gnu_arm_embedded_toolchain/bin/../lib/gcc/arm-none-eabi/9.3.1/thumb/v6-m/nofp\libgcc.a(_udivsi3.o)
 .ARM.attributes
                0x00000252       0x1e c:/program files (x86)/gnu_arm_embedded_toolchain/bin/../lib/gcc/arm-none-eabi/9.3.1/thumb/v6-m/nofp\libgcc.a(_divsi3.o)
 .ARM.attributes
                0x00000270       0x1e c:/program files (x86)/gnu_arm_embedded_toolchain/bin/../lib/gcc/arm-none-eabi/9.3.1/thumb/v6-m/nofp\libgcc.a(_dvmd_tls.o)
 .ARM.attributes
                0x0000028e       0x2c c:/program files (x86)/gnu_arm_embedded_toolchain/bin/../lib/gcc/arm-none-eabi/9.3.1/../../../../arm-none-eabi/lib/thumb/v6-m/nofp\libc_nano.a(lib_a-init.o)
 .ARM.attributes
                0x000002ba       0x2c c:/program files (x86)/gnu_arm_embedded_toolchain/bin/../lib/gcc/arm-none-eabi/9.3.1/../../../../arm-none-eabi/lib/thumb/v6-m/nofp\libc_nano.a(lib_a-memset.o)
 .ARM.attributes
                0x000002e6       0x1e c:/program files (x86)/gnu_arm_embedded_toolchain/bin/../lib/gcc/arm-none-eabi/9.3.1/thumb/v6-m/nofp/crtn.o

.comment        0x00000000       0x4c
 .comment       0x00000000       0x4c Output/startup_samc21.o
                                 0x4d (size before relaxing)
 .comment       0x0000004c       0x4d Output/system_samc21.o
 .comment       0x0000004c       0x4d Output/ADC_Driver.o
 .comment       0x0000004c       0x4d Output/GPIO_Driver.o
 .comment       0x0000004c       0x4d Output/MCAN_Driver.o
 .comment       0x0000004c       0x4d Output/SERCOM_Driver.o
 .comment       0x0000004c       0x4d Output/SYSTEM_Driver.o
 .comment       0x0000004c       0x4d Output/MCAN_Config.o
 .comment       0x0000004c       0x4d Output/main.o
 .comment       0x0000004c       0x4d Output/CommSystem.o
 .comment       0x0000004c       0x4d Output/PdbPowerMonitor.o

.debug_info     0x00000000    0x1d4a9
 .debug_info    0x00000000      0x4e7 Output/startup_samc21.o
 .debug_info    0x000004e7     0x1115 Output/system_samc21.o
 .debug_info    0x000015fc     0x1ec7 Output/ADC_Driver.o
 .debug_info    0x000034c3     0x19f6 Output/GPIO_Driver.o
 .debug_info    0x00004eb9     0x41a1 Output/MCAN_Driver.o
 .debug_info    0x0000905a     0x349d Output/SERCOM_Driver.o
 .debug_info    0x0000c4f7     0x14d0 Output/SYSTEM_Driver.o
 .debug_info    0x0000d9c7     0x3335 Output/MCAN_Config.o
 .debug_info    0x00010cfc     0x3382 Output/main.o
 .debug_info    0x0001407e     0x385a Output/CommSystem.o
 .debug_info    0x000178d8     0x5bd1 Output/PdbPowerMonitor.o

.debug_abbrev   0x00000000     0x1af8
 .debug_abbrev  0x00000000      0x15c Output/startup_samc21.o
 .debug_abbrev  0x0000015c      0x16e Output/system_samc21.o
 .debug_abbrev  0x000002ca      0x203 Output/ADC_Driver.o
 .debug_abbrev  0x000004cd      0x2f9 Output/GPIO_Driver.o
 .debug_abbrev  0x000007c6      0x2c8 Output/MCAN_Driver.o
 .debug_abbrev  0x00000a8e      0x334 Output/SERCOM_Driver.o
 .debug_abbrev  0x00000dc2      0x33b Output/SYSTEM_Driver.o
 .debug_abbrev  0x000010fd      0x1b7 Output/MCAN_Config.o
 .debug_abbrev  0x000012b4      0x1e5 Output/main.o
 .debug_abbrev  0x00001499      0x314 Output/CommSystem.o
 .debug_abbrev  0x000017ad      0x34b Output/PdbPowerMonitor.o

.debug_loc      0x00000000     0x217b
 .debug_loc     0x00000000       0x8b Output/startup_samc21.o
 .debug_loc     0x0000008b      0x376 Output/ADC_Driver.o
 .debug_loc     0x00000401      0x37f Output/GPIO_Driver.o
 .debug_loc     0x00000780      0xac1 Output/MCAN_Driver.o
 .debug_loc     0x00001241      0xbfd Output/SERCOM_Driver.o
 .debug_loc     0x00001e3e      0x1e5 Output/SYSTEM_Driver.o
 .debug_loc     0x00002023       0xe0 Output/CommSystem.o
 .debug_loc     0x00002103       0x78 Output/PdbPowerMonitor.o

.debug_aranges  0x00000000      0x380
 .debug_aranges
                0x00000000       0x28 Output/startup_samc21.o
 .debug_aranges
                0x00000028       0x28 Output/system_samc21.o
 .debug_aranges
                0x00000050       0x70 Output/ADC_Driver.o
 .debug_aranges
                0x000000c0       0x48 Output/GPIO_Driver.o
 .debug_aranges
                0x00000108       0x68 Output/MCAN_Driver.o
 .debug_aranges
                0x00000170       0xd8 Output/SERCOM_Driver.o
 .debug_aranges
                0x00000248       0x68 Output/SYSTEM_Driver.o
 .debug_aranges
                0x000002b0       0x18 Output/MCAN_Config.o
 .debug_aranges
                0x000002c8       0x20 Output/main.o
 .debug_aranges
                0x000002e8       0x48 Output/CommSystem.o
 .debug_aranges
                0x00000330       0x50 Output/PdbPowerMonitor.o

.debug_ranges   0x00000000      0x2e0
 .debug_ranges  0x00000000       0x18 Output/startup_samc21.o
 .debug_ranges  0x00000018       0x18 Output/system_samc21.o
 .debug_ranges  0x00000030       0x78 Output/ADC_Driver.o
 .debug_ranges  0x000000a8       0x38 Output/GPIO_Driver.o
 .debug_ranges  0x000000e0       0x58 Output/MCAN_Driver.o
 .debug_ranges  0x00000138       0xc8 Output/SERCOM_Driver.o
 .debug_ranges  0x00000200       0x58 Output/SYSTEM_Driver.o
 .debug_ranges  0x00000258       0x10 Output/main.o
 .debug_ranges  0x00000268       0x38 Output/CommSystem.o
 .debug_ranges  0x000002a0       0x40 Output/PdbPowerMonitor.o

.debug_macro    0x00000000    0x17dcb
 .debug_macro   0x00000000      0x3ba Output/startup_samc21.o
 .debug_macro   0x000003ba      0xa72 Output/startup_samc21.o
 .debug_macro   0x00000e2c       0x22 Output/startup_samc21.o
 .debug_macro   0x00000e4e       0x8e Output/startup_samc21.o
 .debug_macro   0x00000edc       0x51 Output/startup_samc21.o
 .debug_macro   0x00000f2d      0x103 Output/startup_samc21.o
 .debug_macro   0x00001030       0x6a Output/startup_samc21.o
 .debug_macro   0x0000109a      0x1df Output/startup_samc21.o
 .debug_macro   0x00001279       0x39 Output/startup_samc21.o
 .debug_macro   0x000012b2       0x1c Output/startup_samc21.o
 .debug_macro   0x000012ce       0x22 Output/startup_samc21.o
 .debug_macro   0x000012f0       0xd7 Output/startup_samc21.o
 .debug_macro   0x000013c7      0x4da Output/startup_samc21.o
 .debug_macro   0x000018a1      0x11f Output/startup_samc21.o
 .debug_macro   0x000019c0      0x897 Output/startup_samc21.o
 .debug_macro   0x00002257      0x8c0 Output/startup_samc21.o
 .debug_macro   0x00002b17     0x2d61 Output/startup_samc21.o
 .debug_macro   0x00005878      0x21e Output/startup_samc21.o
 .debug_macro   0x00005a96      0x282 Output/startup_samc21.o
 .debug_macro   0x00005d18      0x130 Output/startup_samc21.o
 .debug_macro   0x00005e48      0xd32 Output/startup_samc21.o
 .debug_macro   0x00006b7a      0x61f Output/startup_samc21.o
 .debug_macro   0x00007199      0x5be Output/startup_samc21.o
 .debug_macro   0x00007757      0x824 Output/startup_samc21.o
 .debug_macro   0x00007f7b      0x172 Output/startup_samc21.o
 .debug_macro   0x000080ed      0x306 Output/startup_samc21.o
 .debug_macro   0x000083f3      0x55f Output/startup_samc21.o
 .debug_macro   0x00008952      0x421 Output/startup_samc21.o
 .debug_macro   0x00008d73      0x21c Output/startup_samc21.o
 .debug_macro   0x00008f8f      0x719 Output/startup_samc21.o
 .debug_macro   0x000096a8      0x5ab Output/startup_samc21.o
 .debug_macro   0x00009c53      0x335 Output/startup_samc21.o
 .debug_macro   0x00009f88      0x68d Output/startup_samc21.o
 .debug_macro   0x0000a615       0xc4 Output/startup_samc21.o
 .debug_macro   0x0000a6d9      0x340 Output/startup_samc21.o
 .debug_macro   0x0000aa19       0x6a Output/startup_samc21.o
 .debug_macro   0x0000aa83     0x124b Output/startup_samc21.o
 .debug_macro   0x0000bcce      0x5a5 Output/startup_samc21.o
 .debug_macro   0x0000c273      0xfc4 Output/startup_samc21.o
 .debug_macro   0x0000d237      0x59e Output/startup_samc21.o
 .debug_macro   0x0000d7d5      0x8ae Output/startup_samc21.o
 .debug_macro   0x0000e083     0x19be Output/startup_samc21.o
 .debug_macro   0x0000fa41      0x39c Output/startup_samc21.o
 .debug_macro   0x0000fddd      0x36a Output/startup_samc21.o
 .debug_macro   0x00010147       0x94 Output/startup_samc21.o
 .debug_macro   0x000101db       0xac Output/startup_samc21.o
 .debug_macro   0x00010287       0xac Output/startup_samc21.o
 .debug_macro   0x00010333      0x149 Output/startup_samc21.o
 .debug_macro   0x0001047c      0x149 Output/startup_samc21.o
 .debug_macro   0x000105c5       0x4c Output/startup_samc21.o
 .debug_macro   0x00010611       0x58 Output/startup_samc21.o
 .debug_macro   0x00010669       0x3a Output/startup_samc21.o
 .debug_macro   0x000106a3       0xd6 Output/startup_samc21.o
 .debug_macro   0x00010779       0xb8 Output/startup_samc21.o
 .debug_macro   0x00010831       0x64 Output/startup_samc21.o
 .debug_macro   0x00010895      0x5d7 Output/startup_samc21.o
 .debug_macro   0x00010e6c       0x4c Output/startup_samc21.o
 .debug_macro   0x00010eb8      0x1be Output/startup_samc21.o
 .debug_macro   0x00011076      0x184 Output/startup_samc21.o
 .debug_macro   0x000111fa       0x52 Output/startup_samc21.o
 .debug_macro   0x0001124c       0xa0 Output/startup_samc21.o
 .debug_macro   0x000112ec       0xd6 Output/startup_samc21.o
 .debug_macro   0x000113c2       0x94 Output/startup_samc21.o
 .debug_macro   0x00011456       0x4c Output/startup_samc21.o
 .debug_macro   0x000114a2       0x64 Output/startup_samc21.o
 .debug_macro   0x00011506       0x22 Output/startup_samc21.o
 .debug_macro   0x00011528      0x16c Output/startup_samc21.o
 .debug_macro   0x00011694       0x2e Output/startup_samc21.o
 .debug_macro   0x000116c2       0x16 Output/startup_samc21.o
 .debug_macro   0x000116d8       0xd6 Output/startup_samc21.o
 .debug_macro   0x000117ae       0xa0 Output/startup_samc21.o
 .debug_macro   0x0001184e      0x133 Output/startup_samc21.o
 .debug_macro   0x00011981      0x133 Output/startup_samc21.o
 .debug_macro   0x00011ab4      0x133 Output/startup_samc21.o
 .debug_macro   0x00011be7      0x133 Output/startup_samc21.o
 .debug_macro   0x00011d1a      0x133 Output/startup_samc21.o
 .debug_macro   0x00011e4d      0x133 Output/startup_samc21.o
 .debug_macro   0x00011f80       0x4c Output/startup_samc21.o
 .debug_macro   0x00011fcc       0xfa Output/startup_samc21.o
 .debug_macro   0x000120c6       0xfa Output/startup_samc21.o
 .debug_macro   0x000121c0       0xfa Output/startup_samc21.o
 .debug_macro   0x000122ba       0xfa Output/startup_samc21.o
 .debug_macro   0x000123b4       0xfa Output/startup_samc21.o
 .debug_macro   0x000124ae      0x124 Output/startup_samc21.o
 .debug_macro   0x000125d2       0xfa Output/startup_samc21.o
 .debug_macro   0x000126cc       0xee Output/startup_samc21.o
 .debug_macro   0x000127ba       0x76 Output/startup_samc21.o
 .debug_macro   0x00012830       0x3a Output/startup_samc21.o
 .debug_macro   0x0001286a      0x46b Output/startup_samc21.o
 .debug_macro   0x00012cd5     0x1de3 Output/startup_samc21.o
 .debug_macro   0x00014ab8       0x82 Output/startup_samc21.o
 .debug_macro   0x00014b3a      0x3c6 Output/system_samc21.o
 .debug_macro   0x00014f00      0x413 Output/ADC_Driver.o
 .debug_macro   0x00015313       0x22 Output/ADC_Driver.o
 .debug_macro   0x00015335       0x3f Output/ADC_Driver.o
 .debug_macro   0x00015374      0x1a3 Output/ADC_Driver.o
 .debug_macro   0x00015517       0x2e Output/ADC_Driver.o
 .debug_macro   0x00015545      0x413 Output/GPIO_Driver.o
 .debug_macro   0x00015958       0xb8 Output/GPIO_Driver.o
 .debug_macro   0x00015a10      0x431 Output/MCAN_Driver.o
 .debug_macro   0x00015e41       0x58 Output/MCAN_Driver.o
 .debug_macro   0x00015e99      0x250 Output/MCAN_Driver.o
 .debug_macro   0x000160e9       0x70 Output/MCAN_Driver.o
 .debug_macro   0x00016159      0x419 Output/SERCOM_Driver.o
 .debug_macro   0x00016572       0x22 Output/SERCOM_Driver.o
 .debug_macro   0x00016594      0x413 Output/SYSTEM_Driver.o
 .debug_macro   0x000169a7       0x28 Output/SYSTEM_Driver.o
 .debug_macro   0x000169cf      0x431 Output/MCAN_Config.o
 .debug_macro   0x00016e00      0x462 Output/main.o
 .debug_macro   0x00017262       0xbe Output/main.o
 .debug_macro   0x00017320       0x5e Output/main.o
 .debug_macro   0x0001737e       0x28 Output/main.o
 .debug_macro   0x000173a6       0x2e Output/main.o
 .debug_macro   0x000173d4      0x477 Output/CommSystem.o
 .debug_macro   0x0001784b       0x40 Output/CommSystem.o
 .debug_macro   0x0001788b      0x540 Output/PdbPowerMonitor.o

.debug_line     0x00000000     0x6de0
 .debug_line    0x00000000      0x697 Output/startup_samc21.o
 .debug_line    0x00000697      0x65d Output/system_samc21.o
 .debug_line    0x00000cf4      0xc31 Output/ADC_Driver.o
 .debug_line    0x00001925      0x9a9 Output/GPIO_Driver.o
 .debug_line    0x000022ce      0xe48 Output/MCAN_Driver.o
 .debug_line    0x00003116      0xf09 Output/SERCOM_Driver.o
 .debug_line    0x0000401f      0x9f7 Output/SYSTEM_Driver.o
 .debug_line    0x00004a16      0x6ab Output/MCAN_Config.o
 .debug_line    0x000050c1      0x73d Output/main.o
 .debug_line    0x000057fe      0x952 Output/CommSystem.o
 .debug_line    0x00006150      0xc90 Output/PdbPowerMonitor.o

.debug_str      0x00000000    0x87c58
 .debug_str     0x00000000    0x81c1f Output/startup_samc21.o
                              0x82628 (size before relaxing)
 .debug_str     0x00081c1f      0x545 Output/system_samc21.o
                              0x827a1 (size before relaxing)
 .debug_str     0x00082164     0x16a1 Output/ADC_Driver.o
                              0x83a47 (size before relaxing)
 .debug_str     0x00083805      0x9ab Output/GPIO_Driver.o
                              0x83611 (size before relaxing)
 .debug_str     0x000841b0     0x271a Output/MCAN_Driver.o
                              0x85281 (size before relaxing)
 .debug_str     0x000868ca      0x9ba Output/SERCOM_Driver.o
                              0x836aa (size before relaxing)
 .debug_str     0x00087284      0x16a Output/SYSTEM_Driver.o
                              0x83182 (size before relaxing)
 .debug_str     0x000873ee       0x45 Output/MCAN_Config.o
                              0x84dbb (size before relaxing)
 .debug_str     0x00087433      0x105 Output/main.o
                              0x8466f (size before relaxing)
 .debug_str     0x00087538      0x28d Output/CommSystem.o
                              0x84965 (size before relaxing)
 .debug_str     0x000877c5      0x493 Output/PdbPowerMonitor.o
                              0x8567e (size before relaxing)

.debug_frame    0x00000000      0x7fc
 .debug_frame   0x00000000       0x38 Output/startup_samc21.o
 .debug_frame   0x00000038       0x30 Output/system_samc21.o
 .debug_frame   0x00000068       0xe0 Output/ADC_Driver.o
 .debug_frame   0x00000148       0xa0 Output/GPIO_Driver.o
 .debug_frame   0x000001e8       0xf0 Output/MCAN_Driver.o
 .debug_frame   0x000002d8      0x258 Output/SERCOM_Driver.o
 .debug_frame   0x00000530       0xc0 Output/SYSTEM_Driver.o
 .debug_frame   0x000005f0       0x28 Output/main.o
 .debug_frame   0x00000618       0xb0 Output/CommSystem.o
 .debug_frame   0x000006c8       0xa8 Output/PdbPowerMonitor.o
 .debug_frame   0x00000770       0x20 c:/program files (x86)/gnu_arm_embedded_toolchain/bin/../lib/gcc/arm-none-eabi/9.3.1/thumb/v6-m/nofp\libgcc.a(_udivsi3.o)
 .debug_frame   0x00000790       0x20 c:/program files (x86)/gnu_arm_embedded_toolchain/bin/../lib/gcc/arm-none-eabi/9.3.1/thumb/v6-m/nofp\libgcc.a(_divsi3.o)
 .debug_frame   0x000007b0       0x2c c:/program files (x86)/gnu_arm_embedded_toolchain/bin/../lib/gcc/arm-none-eabi/9.3.1/../../../../arm-none-eabi/lib/thumb/v6-m/nofp\libc_nano.a(lib_a-init.o)
 .debug_frame   0x000007dc       0x20 c:/program files (x86)/gnu_arm_embedded_toolchain/bin/../lib/gcc/arm-none-eabi/9.3.1/../../../../arm-none-eabi/lib/thumb/v6-m/nofp\libc_nano.a(lib_a-memset.o)

Cross Reference Table

Symbol                                            File
AC_Handler                                        Output/startup_samc21.o
ADC0_Handler                                      Output/startup_samc21.o
ADC1_Handler                                      Output/startup_samc21.o
ADC_ChangeReference                               Output/ADC_Driver.o
ADC_Initialize                                    Output/ADC_Driver.o
                                                  Output/PdbPowerMonitor.o
ADC_SetAveraging                                  Output/ADC_Driver.o
ADC_SetDifferentialChannel                        Output/ADC_Driver.o
ADC_SetEvents                                     Output/ADC_Driver.o
ADC_SetSequence                                   Output/ADC_Driver.o
ADC_SetSingleEndedChannel                         Output/ADC_Driver.o
                                                  Output/PdbPowerMonitor.o
ADC_SetWindowMonitor                              Output/ADC_Driver.o
ADC_StartConversion                               Output/ADC_Driver.o
                                                  Output/PdbPowerMonitor.o
ADC_StopConversion                                Output/ADC_Driver.o
CAN0_Handler                                      Output/startup_samc21.o
CAN1_Handler                                      Output/startup_samc21.o
CommSystem_ComposeMessage                         Output/CommSystem.o
CommSystem_Initialize                             Output/CommSystem.o
                                                  Output/main.o
CommSystem_SendData                               Output/CommSystem.o
                                                  Output/PdbPowerMonitor.o
CommSystem_SendFault                              Output/CommSystem.o
                                                  Output/PdbPowerMonitor.o
CommSystem_SendStatus                             Output/CommSystem.o
CommSystem_Task                                   Output/CommSystem.o
                                                  Output/main.o
CreateStaticFifoBuffer                            Output/fifobuffer.o
DAC_Handler                                       Output/startup_samc21.o
DMAC_Handler                                      Output/startup_samc21.o
Dummy_Handler                                     Output/startup_samc21.o
ECUOnline                                         Output/CommSystem.o
EIC_Handler                                       Output/PdbPowerMonitor.o
                                                  Output/startup_samc21.o
EVSYS_Handler                                     Output/startup_samc21.o
EXTINT_ConfigureChannel                           Output/GPIO_Driver.o
EXTINT_ConfigureNMI                               Output/GPIO_Driver.o
EXTINT_Initialize                                 Output/GPIO_Driver.o
FREQM_Handler                                     Output/startup_samc21.o
FifoBuffer_Flush                                  Output/fifobuffer.o
FifoBuffer_FlushBytes                             Output/fifobuffer.o
FifoBuffer_GetLenght                              Output/fifobuffer.o
FifoBuffer_GetSize                                Output/fifobuffer.o
FifoBuffer_PeekBytesUntil                         Output/fifobuffer.o
FifoBuffer_ReadByte                               Output/fifobuffer.o
FifoBuffer_ReadByteFromISR                        Output/fifobuffer.o
                                                  Output/SERCOM_Driver.o
FifoBuffer_ReadBytes                              Output/fifobuffer.o
FifoBuffer_SetLockFunc                            Output/fifobuffer.o
                                                  Output/SERCOM_Driver.o
FifoBuffer_WriteByte                              Output/fifobuffer.o
FifoBuffer_WriteByteFromISR                       Output/fifobuffer.o
                                                  Output/SERCOM_Driver.o
FifoBuffer_WriteBytes                             Output/fifobuffer.o
FifoBuffer_WriteString                            Output/fifobuffer.o
GPIO_GetPinState                                  Output/GPIO_Driver.o
                                                  Output/PdbPowerMonitor.o
GPIO_SetPinMode                                   Output/GPIO_Driver.o
                                                  Output/PdbPowerMonitor.o
                                                  Output/CommSystem.o
GPIO_SetPinMux                                    Output/GPIO_Driver.o
                                                  Output/PdbPowerMonitor.o
                                                  Output/CommSystem.o
HardFault_Handler                                 Output/startup_samc21.o
I2C_Initialize                                    Output/SERCOM_Driver.o
I2C_Read                                          Output/SERCOM_Driver.o
I2C_ReadRegisterBA                                Output/SERCOM_Driver.o
I2C_ReadRegisterWA                                Output/SERCOM_Driver.o
I2C_SetMode                                       Output/SERCOM_Driver.o
I2C_Write                                         Output/SERCOM_Driver.o
I2C_WriteRegisterBA                               Output/SERCOM_Driver.o
I2C_WriteRegisterWA                               Output/SERCOM_Driver.o
IVREF_Setup                                       Output/ADC_Driver.o
                                                  Output/PdbPowerMonitor.o
MCAN0                                             Output/MCAN_Driver.o
                                                  Output/CommSystem.o
MCAN0_Config                                      Output/MCAN_Config.o
                                                  Output/MCAN_Driver.o
MCAN_ChangeMode                                   Output/MCAN_Driver.o
                                                  Output/CommSystem.o
MCAN_ConfigureBitTimings                          Output/MCAN_Driver.o
MCAN_ConfigureExtendedIdGlobalMask                Output/MCAN_Driver.o
MCAN_ConfigureGlobalFilter                        Output/MCAN_Driver.o
MCAN_GetCurrentMode                               Output/MCAN_Driver.o
MCAN_Initialize                                   Output/MCAN_Driver.o
                                                  Output/CommSystem.o
MCAN_LoadExtendedFilter                           Output/MCAN_Driver.o
MCAN_LoadStandardFilter                           Output/MCAN_Driver.o
MCAN_ReadFIFOMessage                              Output/MCAN_Driver.o
                                                  Output/CommSystem.o
MCAN_TransmitMessageFIFO                          Output/MCAN_Driver.o
                                                  Output/CommSystem.o
NVMCTRL_Handler                                   Output/startup_samc21.o
NonMaskableInt_Handler                            Output/startup_samc21.o
PTC_Handler                                       Output/startup_samc21.o
PdbPwrMonData                                     Output/PdbPowerMonitor.o
PdbPwrMon_ADC                                     Output/PdbPowerMonitor.o
PdbPwrMon_FaultControl                            Output/PdbPowerMonitor.o
PdbPwrMon_GetData                                 Output/PdbPowerMonitor.o
                                                  Output/CommSystem.o
PdbPwrMon_Initialize                              Output/PdbPowerMonitor.o
                                                  Output/main.o
PdbPwrMon_Task                                    Output/PdbPowerMonitor.o
                                                  Output/main.o
PdbPwrMon_eFuseControl                            Output/PdbPowerMonitor.o
PendSV_Handler                                    Output/startup_samc21.o
RTC_Handler                                       Output/startup_samc21.o
Reset_Handler                                     Output/startup_samc21.o
SDADC_Handler                                     Output/startup_samc21.o
SERCOM0_Handler                                   Output/SERCOM_Driver.o
                                                  Output/startup_samc21.o
SERCOM1_Handler                                   Output/SERCOM_Driver.o
                                                  Output/startup_samc21.o
SERCOM2_Handler                                   Output/SERCOM_Driver.o
                                                  Output/startup_samc21.o
SERCOM3_Handler                                   Output/SERCOM_Driver.o
                                                  Output/startup_samc21.o
SERCOM4_Handler                                   Output/SERCOM_Driver.o
                                                  Output/startup_samc21.o
SERCOM5_Handler                                   Output/SERCOM_Driver.o
                                                  Output/startup_samc21.o
SVCall_Handler                                    Output/startup_samc21.o
SYSTEM_ClearSysTickCallbacks                      Output/SYSTEM_Driver.o
SYSTEM_GetSysTickCount                            Output/SYSTEM_Driver.o
                                                  Output/PdbPowerMonitor.o
                                                  Output/CommSystem.o
SYSTEM_Handler                                    Output/startup_samc21.o
SYSTEM_IncrementSysTickCount                      Output/SYSTEM_Driver.o
SYSTEM_InitalizeSysTick                           Output/SYSTEM_Driver.o
                                                  Output/main.o
SYSTEM_InitializeClocks                           Output/SYSTEM_Driver.o
                                                  Output/main.o
SYSTEM_IsClockSourceAvailable                     Output/SYSTEM_Driver.o
                                                  Output/SERCOM_Driver.o
                                                  Output/GPIO_Driver.o
                                                  Output/ADC_Driver.o
SYSTEM_RegisterSysTickCallback                    Output/SYSTEM_Driver.o
SYSTEM_UnregisterSysTickCallback                  Output/SYSTEM_Driver.o
SYSTEM_UpdateSysTickCount                         Output/SYSTEM_Driver.o
SysTickCallbacks                                  Output/SYSTEM_Driver.o
SysTick_Handler                                   Output/SYSTEM_Driver.o
                                                  Output/startup_samc21.o
SystemCoreClock                                   Output/system_samc21.o
                                                  Output/SYSTEM_Driver.o
                                                  Output/SERCOM_Driver.o
SystemCoreClockUpdate                             Output/system_samc21.o
SystemInit                                        Output/system_samc21.o
                                                  Output/startup_samc21.o
TC0_Handler                                       Output/startup_samc21.o
TC1_Handler                                       Output/startup_samc21.o
TC2_Handler                                       Output/startup_samc21.o
TC3_Handler                                       Output/startup_samc21.o
TC4_Handler                                       Output/startup_samc21.o
TCC0_Handler                                      Output/startup_samc21.o
TCC1_Handler                                      Output/startup_samc21.o
TCC2_Handler                                      Output/startup_samc21.o
TSENS_Handler                                     Output/startup_samc21.o
UART_Initialize                                   Output/SERCOM_Driver.o
UART_LinkBuffers                                  Output/SERCOM_Driver.o
UART_RxLock                                       Output/SERCOM_Driver.o
UART_RxUnlock                                     Output/SERCOM_Driver.o
UART_SetMode                                      Output/SERCOM_Driver.o
UART_TxLock                                       Output/SERCOM_Driver.o
UART_TxUnlock                                     Output/SERCOM_Driver.o
WDT_Handler                                       Output/startup_samc21.o
_MCAN0_message_ram                                Output/MCAN_Driver.o
__aeabi_idiv                                      c:/program files (x86)/gnu_arm_embedded_toolchain/bin/../lib/gcc/arm-none-eabi/9.3.1/thumb/v6-m/nofp\libgcc.a(_divsi3.o)
                                                  Output/PdbPowerMonitor.o
__aeabi_idiv0                                     c:/program files (x86)/gnu_arm_embedded_toolchain/bin/../lib/gcc/arm-none-eabi/9.3.1/thumb/v6-m/nofp\libgcc.a(_dvmd_tls.o)
                                                  c:/program files (x86)/gnu_arm_embedded_toolchain/bin/../lib/gcc/arm-none-eabi/9.3.1/thumb/v6-m/nofp\libgcc.a(_divsi3.o)
                                                  c:/program files (x86)/gnu_arm_embedded_toolchain/bin/../lib/gcc/arm-none-eabi/9.3.1/thumb/v6-m/nofp\libgcc.a(_udivsi3.o)
__aeabi_idivmod                                   c:/program files (x86)/gnu_arm_embedded_toolchain/bin/../lib/gcc/arm-none-eabi/9.3.1/thumb/v6-m/nofp\libgcc.a(_divsi3.o)
__aeabi_ldiv0                                     c:/program files (x86)/gnu_arm_embedded_toolchain/bin/../lib/gcc/arm-none-eabi/9.3.1/thumb/v6-m/nofp\libgcc.a(_dvmd_tls.o)
                                                  c:/program files (x86)/gnu_arm_embedded_toolchain/bin/../lib/gcc/arm-none-eabi/9.3.1/thumb/v6-m/nofp\libgcc.a(_aeabi_uldivmod.o)
__aeabi_uidiv                                     c:/program files (x86)/gnu_arm_embedded_toolchain/bin/../lib/gcc/arm-none-eabi/9.3.1/thumb/v6-m/nofp\libgcc.a(_udivsi3.o)
                                                  Output/SYSTEM_Driver.o
                                                  Output/SERCOM_Driver.o
                                                  Output/printf.o
__aeabi_uidivmod                                  c:/program files (x86)/gnu_arm_embedded_toolchain/bin/../lib/gcc/arm-none-eabi/9.3.1/thumb/v6-m/nofp\libgcc.a(_udivsi3.o)
                                                  Output/printf.o
__aeabi_uldivmod                                  c:/program files (x86)/gnu_arm_embedded_toolchain/bin/../lib/gcc/arm-none-eabi/9.3.1/thumb/v6-m/nofp\libgcc.a(_aeabi_uldivmod.o)
                                                  Output/printf.o
__bss_end__                                       c:/program files (x86)/gnu_arm_embedded_toolchain/bin/../lib/gcc/arm-none-eabi/9.3.1/../../../../arm-none-eabi/lib/thumb/v6-m/nofp/crt0.o
__bss_start__                                     c:/program files (x86)/gnu_arm_embedded_toolchain/bin/../lib/gcc/arm-none-eabi/9.3.1/../../../../arm-none-eabi/lib/thumb/v6-m/nofp/crt0.o
__call_exitprocs                                  c:/program files (x86)/gnu_arm_embedded_toolchain/bin/../lib/gcc/arm-none-eabi/9.3.1/../../../../arm-none-eabi/lib/thumb/v6-m/nofp\libc_nano.a(lib_a-exit.o)
__clzdi2                                          c:/program files (x86)/gnu_arm_embedded_toolchain/bin/../lib/gcc/arm-none-eabi/9.3.1/thumb/v6-m/nofp\libgcc.a(_clzdi2.o)
                                                  c:/program files (x86)/gnu_arm_embedded_toolchain/bin/../lib/gcc/arm-none-eabi/9.3.1/thumb/v6-m/nofp\libgcc.a(_udivmoddi4.o)
__clzsi2                                          c:/program files (x86)/gnu_arm_embedded_toolchain/bin/../lib/gcc/arm-none-eabi/9.3.1/thumb/v6-m/nofp\libgcc.a(_clzsi2.o)
                                                  c:/program files (x86)/gnu_arm_embedded_toolchain/bin/../lib/gcc/arm-none-eabi/9.3.1/thumb/v6-m/nofp\libgcc.a(_clzdi2.o)
__deregister_frame_info                           c:/program files (x86)/gnu_arm_embedded_toolchain/bin/../lib/gcc/arm-none-eabi/9.3.1/thumb/v6-m/nofp/crtbegin.o
__divsi3                                          c:/program files (x86)/gnu_arm_embedded_toolchain/bin/../lib/gcc/arm-none-eabi/9.3.1/thumb/v6-m/nofp\libgcc.a(_divsi3.o)
__dso_handle                                      c:/program files (x86)/gnu_arm_embedded_toolchain/bin/../lib/gcc/arm-none-eabi/9.3.1/thumb/v6-m/nofp/crtbegin.o
__init_array_end                                  c:/program files (x86)/gnu_arm_embedded_toolchain/bin/../lib/gcc/arm-none-eabi/9.3.1/../../../../arm-none-eabi/lib/thumb/v6-m/nofp\libc_nano.a(lib_a-init.o)
__init_array_start                                c:/program files (x86)/gnu_arm_embedded_toolchain/bin/../lib/gcc/arm-none-eabi/9.3.1/../../../../arm-none-eabi/lib/thumb/v6-m/nofp\libc_nano.a(lib_a-init.o)
__libc_fini_array                                 c:/program files (x86)/gnu_arm_embedded_toolchain/bin/../lib/gcc/arm-none-eabi/9.3.1/../../../../arm-none-eabi/lib/thumb/v6-m/nofp/crt0.o
__libc_init_array                                 c:/program files (x86)/gnu_arm_embedded_toolchain/bin/../lib/gcc/arm-none-eabi/9.3.1/../../../../arm-none-eabi/lib/thumb/v6-m/nofp\libc_nano.a(lib_a-init.o)
                                                  Output/startup_samc21.o
                                                  c:/program files (x86)/gnu_arm_embedded_toolchain/bin/../lib/gcc/arm-none-eabi/9.3.1/../../../../arm-none-eabi/lib/thumb/v6-m/nofp/crt0.o
__preinit_array_end                               c:/program files (x86)/gnu_arm_embedded_toolchain/bin/../lib/gcc/arm-none-eabi/9.3.1/../../../../arm-none-eabi/lib/thumb/v6-m/nofp\libc_nano.a(lib_a-init.o)
__preinit_array_start                             c:/program files (x86)/gnu_arm_embedded_toolchain/bin/../lib/gcc/arm-none-eabi/9.3.1/../../../../arm-none-eabi/lib/thumb/v6-m/nofp\libc_nano.a(lib_a-init.o)
__register_frame_info                             c:/program files (x86)/gnu_arm_embedded_toolchain/bin/../lib/gcc/arm-none-eabi/9.3.1/thumb/v6-m/nofp/crtbegin.o
__sf_fake_stderr                                  c:/program files (x86)/gnu_arm_embedded_toolchain/bin/../lib/gcc/arm-none-eabi/9.3.1/../../../../arm-none-eabi/lib/thumb/v6-m/nofp\libc_nano.a(lib_a-impure.o)
__sf_fake_stdin                                   c:/program files (x86)/gnu_arm_embedded_toolchain/bin/../lib/gcc/arm-none-eabi/9.3.1/../../../../arm-none-eabi/lib/thumb/v6-m/nofp\libc_nano.a(lib_a-impure.o)
__sf_fake_stdout                                  c:/program files (x86)/gnu_arm_embedded_toolchain/bin/../lib/gcc/arm-none-eabi/9.3.1/../../../../arm-none-eabi/lib/thumb/v6-m/nofp\libc_nano.a(lib_a-impure.o)
__stack                                           c:/program files (x86)/gnu_arm_embedded_toolchain/bin/../lib/gcc/arm-none-eabi/9.3.1/../../../../arm-none-eabi/lib/thumb/v6-m/nofp/crt0.o
__udivmoddi4                                      c:/program files (x86)/gnu_arm_embedded_toolchain/bin/../lib/gcc/arm-none-eabi/9.3.1/thumb/v6-m/nofp\libgcc.a(_udivmoddi4.o)
                                                  c:/program files (x86)/gnu_arm_embedded_toolchain/bin/../lib/gcc/arm-none-eabi/9.3.1/thumb/v6-m/nofp\libgcc.a(_aeabi_uldivmod.o)
__udivsi3                                         c:/program files (x86)/gnu_arm_embedded_toolchain/bin/../lib/gcc/arm-none-eabi/9.3.1/thumb/v6-m/nofp\libgcc.a(_udivsi3.o)
_erelocate                                        Output/startup_samc21.o
_estack                                           Output/startup_samc21.o
_etext                                            Output/startup_samc21.o
_exit                                             c:/program files (x86)/gnu_arm_embedded_toolchain/bin/../lib/gcc/arm-none-eabi/9.3.1/../../../../arm-none-eabi/lib/thumb/v6-m/nofp\libc_nano.a(lib_a-exit.o)
_ezero                                            Output/startup_samc21.o
_fini                                             c:/program files (x86)/gnu_arm_embedded_toolchain/bin/../lib/gcc/arm-none-eabi/9.3.1/thumb/v6-m/nofp/crti.o
_global_impure_ptr                                c:/program files (x86)/gnu_arm_embedded_toolchain/bin/../lib/gcc/arm-none-eabi/9.3.1/../../../../arm-none-eabi/lib/thumb/v6-m/nofp\libc_nano.a(lib_a-impure.o)
                                                  c:/program files (x86)/gnu_arm_embedded_toolchain/bin/../lib/gcc/arm-none-eabi/9.3.1/../../../../arm-none-eabi/lib/thumb/v6-m/nofp\libc_nano.a(lib_a-exit.o)
_impure_ptr                                       c:/program files (x86)/gnu_arm_embedded_toolchain/bin/../lib/gcc/arm-none-eabi/9.3.1/../../../../arm-none-eabi/lib/thumb/v6-m/nofp\libc_nano.a(lib_a-impure.o)
_init                                             c:/program files (x86)/gnu_arm_embedded_toolchain/bin/../lib/gcc/arm-none-eabi/9.3.1/thumb/v6-m/nofp/crti.o
                                                  c:/program files (x86)/gnu_arm_embedded_toolchain/bin/../lib/gcc/arm-none-eabi/9.3.1/../../../../arm-none-eabi/lib/thumb/v6-m/nofp\libc_nano.a(lib_a-init.o)
_mainCRTStartup                                   c:/program files (x86)/gnu_arm_embedded_toolchain/bin/../lib/gcc/arm-none-eabi/9.3.1/../../../../arm-none-eabi/lib/thumb/v6-m/nofp/crt0.o
_mcan0_init_extfilters                            Output/MCAN_Config.o
_mcan0_init_stdfilters                            Output/MCAN_Config.o
_putchar                                          Output/printf.o
_sfixed                                           Output/startup_samc21.o
_srelocate                                        Output/startup_samc21.o
_stack_init                                       c:/program files (x86)/gnu_arm_embedded_toolchain/bin/../lib/gcc/arm-none-eabi/9.3.1/../../../../arm-none-eabi/lib/thumb/v6-m/nofp/crt0.o
_start                                            c:/program files (x86)/gnu_arm_embedded_toolchain/bin/../lib/gcc/arm-none-eabi/9.3.1/../../../../arm-none-eabi/lib/thumb/v6-m/nofp/crt0.o
_szero                                            Output/startup_samc21.o
atexit                                            c:/program files (x86)/gnu_arm_embedded_toolchain/bin/../lib/gcc/arm-none-eabi/9.3.1/../../../../arm-none-eabi/lib/thumb/v6-m/nofp/crt0.o
datelFaultTime                                    Output/PdbPowerMonitor.o
datelFaults                                       Output/PdbPowerMonitor.o
ecupcFaultTime                                    Output/PdbPowerMonitor.o
ecupcFaults                                       Output/PdbPowerMonitor.o
exception_table                                   Output/startup_samc21.o
exit                                              c:/program files (x86)/gnu_arm_embedded_toolchain/bin/../lib/gcc/arm-none-eabi/9.3.1/../../../../arm-none-eabi/lib/thumb/v6-m/nofp\libc_nano.a(lib_a-exit.o)
                                                  c:/program files (x86)/gnu_arm_embedded_toolchain/bin/../lib/gcc/arm-none-eabi/9.3.1/../../../../arm-none-eabi/lib/thumb/v6-m/nofp/crt0.o
fctprintf                                         Output/printf.o
hardware_init_hook                                c:/program files (x86)/gnu_arm_embedded_toolchain/bin/../lib/gcc/arm-none-eabi/9.3.1/../../../../arm-none-eabi/lib/thumb/v6-m/nofp/crt0.o
invaFaultTime                                     Output/PdbPowerMonitor.o
invaFaults                                        Output/PdbPowerMonitor.o
invfFaultTime                                     Output/PdbPowerMonitor.o
invfFaults                                        Output/PdbPowerMonitor.o
lastAcqTime                                       Output/PdbPowerMonitor.o
lastExtLedBlinkTime                               Output/PdbPowerMonitor.o
lastStatusMessage                                 Output/CommSystem.o
main                                              Output/main.o
                                                  Output/startup_samc21.o
                                                  c:/program files (x86)/gnu_arm_embedded_toolchain/bin/../lib/gcc/arm-none-eabi/9.3.1/../../../../arm-none-eabi/lib/thumb/v6-m/nofp/crt0.o
memset                                            c:/program files (x86)/gnu_arm_embedded_toolchain/bin/../lib/gcc/arm-none-eabi/9.3.1/../../../../arm-none-eabi/lib/thumb/v6-m/nofp\libc_nano.a(lib_a-memset.o)
                                                  Output/CommSystem.o
                                                  c:/program files (x86)/gnu_arm_embedded_toolchain/bin/../lib/gcc/arm-none-eabi/9.3.1/../../../../arm-none-eabi/lib/thumb/v6-m/nofp/crt0.o
printf_                                           Output/printf.o
safamFaultTime                                    Output/PdbPowerMonitor.o
safamFaults                                       Output/PdbPowerMonitor.o
snprintf_                                         Output/printf.o
software_init_hook                                c:/program files (x86)/gnu_arm_embedded_toolchain/bin/../lib/gcc/arm-none-eabi/9.3.1/../../../../arm-none-eabi/lib/thumb/v6-m/nofp/crt0.o
sprintf_                                          Output/printf.o
uart_isr_handler                                  Output/SERCOM_Driver.o
vprintf_                                          Output/printf.o
vsnprintf_                                        Output/printf.o
